:020000040000FA
:02000000802856
:08000800A000030EA100831605
:1000100003130C1C2328831203130C1C23280C101D
:1000200090010B308F00E0308E000B308F00D63007
:100030008E00AF0A08302F06031D2028AF014B1792
:10004000313090000C1083120313210E8300A00E98
:10005000200E0900820052344534473455344C3464
:100060004134543449344F344E34203441344334D1
:10007000433455344D344D34003454344F344734C4
:100080003D34003443344F344E3453343D34003423
:1000900043344D3444343D340034443441345434D6
:1000A00041343D34003450344E3454343D34003403
:1000B000493452345234433435342D34503454346A
:1000C00031343034303420344C344D3433343534DE
:1000D00020344C344D3433343334353400343634F6
:1000E0003234383472346534673430343634313431
:1000F0003234323436342E34413453344D340034B7
:1001000083018B018A018601850107309F008316D8
:1001100003138C0100308500073086000130810018
:1001200083120313203084008001840A841F9428E2
:10013000831603130830AF009830B0000D30B100C3
:10014000AC30B2000A30AC0083120313CB010512AD
:100150000000861107272925F024F324AA24B413CC
:10016000B6136924FC24AB221C27FF242B30D42295
:100170001C27FF245830D4221C27FF246F30D422A0
:100180001C27CE010230B000D00131309000831620
:1001900003130C14831203133E30C7000B178B1785
:1001A000AA24FC24AB224B1BF428C122FF304E05AD
:1001B0000319D0280B12043050060319E428053027
:1001C00050060319E428EC281C304E060319202A97
:1001D0001D304E060319512A2B304E060319FE28F6
:1001E0002C304E060319F8284B1B6925CE01032934
:1001F0003008FF3E031C0329B00303293008073CE5
:10020000031C0329B00A8312031330080739B00016
:100210000030300603192D29013030060319372923
:1002200002303006031945290330300603196D29C1
:10023000043030060319B329053030060319812A2A
:10024000063030060319812A073030060319CD29FC
:1002500083120313CE01B001D0280000FF246F30B9
:10026000D422C8290D30F4220A30F4220800FF24D9
:10027000D001DE22BB01C8305325831603133F088B
:10028000B5004008B6004E23C829FF240130D00035
:10029000DE220130BB00C83053258316031341080A
:1002A000B5004208B6004E2383120313CB1CC829A5
:1002B0001527C630532546300E25C8305325CB159B
:1002C000831603134708B5004808B6004E2383126F
:1002D00003131527CB10CB11C829FF240230D000FF
:1002E000DE220B250130BB00C830532583160313D3
:1002F0004308B5004408B6000130B7009030B8009C
:100300007926B51F8C29B509B609B60A83120313DD
:100310000330BB00831603134E23831203134B1DBC
:10032000C82915270130BB00C630532546300E259D
:10033000C8305325CB15831603134908B5004A0866
:10034000B6000F30B700A030B8007926B51FAD2930
:10035000B509B609B60A0330BB004E238312031356
:100360004B11CB11C829FF240330D000DE22C63048
:1003700053254A304B1C4E300E250430BB00C8308C
:100380005325831603134508B5004608B6004E23CF
:1003900083120313BB01CE01D0288B13082506302E
:1003A000D000DE22AB22C12201304E06031DDA2925
:1003B0006F271A2A00304E06031DE02977271A2AD4
:1003C00003304E06031DE6297D271A2A02304E0609
:1003D000031DEC2985271A2A05304E06031DF22934
:1003E0008B271A2A04304E06031DF82993271A2A50
:1003F00007304E06031DFE2999271A2A06304E069D
:10040000031D042AA1271A2A09304E06031D0A2AB1
:10041000A7271A2A08304E06031D102AAF271A2ACA
:1004200057304E06031DCE2983120313CE01B001AF
:100430008B17D0281C22CE296924AB22CE010800BC
:1004400001304C06031D812A05303006031D302A79
:10045000831603133008B6002F08B5000A30372A78
:10046000831603133208B6003108B5003230B800E5
:10047000B70167268312031305303006031D472A90
:10048000831603133508AF003608B0004D2A8316D3
:1004900003133508B1003608B20083120313CC01F0
:1004A000812A01304C06031D812A05303006031DC8
:1004B000612A831603133008B6002F08B5000A30EE
:1004C000682A831603133208B6003108B5003230AB
:1004D000B800B70179268312031305303006031DD7
:1004E000782A831603133508AF003608B0007E2A39
:1004F000831603133508B1003608B20083120313C4
:10050000CC01FF24CB1105303006031D892A0430AD
:100510008A2A0530D000DE220130BB00C8305325C6
:1005200005303006031D9C2ACB15831603132F08B4
:10053000B5003008B600A32ACB1183160313310887
:10054000B5003208B6004E2383120313CB111527D2
:10055000BB01CE01D528F3243A089A2438089A24FE
:1005600037089A2420300E2536089A243A300E2572
:1005700035089A243A300E2534089A2420300E2566
:1005800008004B1BD32A061CC12A4B1BD32A061872
:10059000C52A933081000B110310C3230318C52A09
:1005A000F8230318C52A0800A80028082A20003AC2
:1005B0000319DD2A0E25A80AD52A08005008A7002D
:1005C0000310A70DA70DA70DA70DA8012808270741
:1005D000831603139B001C141A08831203130E25A1
:1005E000A80A281EE62A080083120313C600083052
:1005F000C8008613CB26C60C0318002B8613012BCC
:100600008617CB26C80BFB2A8617CB26CB260800DD
:1006100083160313A5003030A200A3006430250226
:10062000031C152BA500A20A0E2B0A302502031C61
:100630001C2BA500A30A152B30302507A400220887
:10064000F422831603132308F422831603132408C9
:10065000F422080083160313A5003030A200A30083
:1006600064302502031C372BA500A20A302B0A3068
:100670002502031C3E2BA500A30A372B303025078B
:10068000A40022080E258316031323080E258316C3
:10069000031324080E258312031308008316031383
:1006A0003508B3003608B400350EF038A800A807A6
:1006B000E23EA900323EAB0033080F39A907A90773
:1006C000AB07E93EAA00AA07AA07340E0F39AA070A
:1006D000AB07AA0DAB0DAB09AB0D34080F39AB0757
:1006E000A80D0730A7000A30AB07AA03031C742B20
:1006F000AA07A903031C782BA907A803031C7C2BBA
:10070000A807A703031C802B831203132B30BB1CE9
:100710008C2B3B1C8C2B2D300E25831603132808A5
:10072000831203130319962B303E972B20300E258E
:1007300083160313290883120313303E0E252C3031
:10074000CB1DA42B3B1D0E25831603132A088312F1
:100750000313303E0E252C30CB19B02B3B1D0E253C
:10076000831603132B0883120313303E0E253B1907
:10077000BE2B64300E2543300E2508006D300E254B
:1007800056300E2508008312031357308400800171
:10079000840A5D300406031DC72BD401D5015730F0
:1007A00084000B1DD12BF2230618672C0B1DD62BB2
:1007B000F223D40A2B3054060319E62B031406182F
:1007C0000310800DD50AD519EF23D62B0310800D09
:1007D000800D800D800D800D800D03100800840AAF
:1007E000D5010800831203130B1125308100080086
:1007F00057308400D601D501DF01DD01CC01CD01E8
:10080000CE01CF01800DD60D800DD60DD50A5A240C
:100810005E19672CDE0CDD0DD601800DD60D800D26
:10082000D60DD50A5A245E19672CDE0CCC0D053086
:10083000A900D601800DD60D800DD60DD50A55190B
:10084000EF235A245E19672CDE0CCD0DA90B192C51
:10085000C0305805031D322CEF23800D800DD50AC2
:100860000130DF000630A900D601800DD60D800DC5
:10087000D60DD50A5519EF235A245E19672CDE0CC4
:10088000CE0DA90B342C5D1C4E175F18482C0800A8
:100890000630A900D601800DD60D800DD60DD50AE3
:1008A0005519EF235A245E19672CDE0CCF0DA90BC6
:1008B0004A2C0800DE01013056060319652C02306F
:1008C00056060319662C5E1508005E140800031412
:1008D000080083120313061300000000000000004C
:1008E0000000000006110000000005158316031328
:1008F0000611831203138E30CC240030CC24073031
:10090000A5008030AD0034308400051100000000E7
:100910000613000000000000051500002D08CC247F
:100920000008CC24840AAD0AAD0AA50B852C05115C
:1009300000000800A200A300A20E0F30A205303074
:1009400022070E252308A2000F30A205303022070F
:100950000E25080006130000051183160313061167
:1009600083120313000000000000000006110000C5
:100970000515BF30CC248316031306158312031309
:1009800034308400DF24DF24DF24DF24DF24DF246D
:10099000DF24051100000800B3000830A40006138E
:1009A0000000331C0611000033180615000000007B
:1009B000000006170000B30CA40BCF2C0800083071
:1009C000A300061300000000800C80130619801796
:1009D0000000061700000000A30BE12C840A0800A9
:1009E00001305325F92E1030E10080305325F926CF
:1009F00020300E25E10BF82C80305325F92E1030D5
:100A0000E100C0305325F92620300E25E10B042DDE
:100A1000C0305325F92E02305325F92E83120313CB
:100A2000E000F2260F3086056008F03986040000E9
:100A3000051400008514DD268510DD260F3086059F
:100A4000600EF039860400008514DD268510DD2651
:100A500008008510000005100000F9260F308605FB
:100A600030308604831603130F3006058600831288
:100A70000313851400008510F926851400008510E5
:100A8000F92685140000851007270F3086052030D1
:100A9000860485140000851028305325083053251E
:100AA0000C3053250630E00007270F30860560081C
:100AB000F039860400000510000085140000851040
:100AC0000F308605600EF03986048514000085100D
:100AD000080083120313BB010612000086120000F7
:100AE0002426831603133230B800B70179260A3062
:100AF000B800B70182265C263508BF003608C00062
:100B00008B133F08B5004008B6003108B700320823
:100B1000B800BD26031C902D000086150000A12DF5
:100B2000831203133F08B5004008B6002C08B80034
:100B3000B70179263108B7003208B800BD2603187E
:100B400086118B170130BB000616000086120000CC
:100B50002426831603133508C1003608C2004D0849
:100B6000B7004E08B80067263508CD003608CE001D
:100B7000AD0A0A302D02031DDC2D8B133508C7008A
:100B80003608C8002F08B7003008B800BD26031C7F
:100B9000CE2D8312031305120000D22D83120313EE
:100BA00005160000000083160313AD01CD01CE0130
:100BB00083120313CB148B17831203130130BB0072
:100BC000061200008616000024268316031309303F
:100BD000B7001A30B80079263508C3003608C400BB
:100BE0004B08B7004C08B80067263508CB0036081C
:100BF000CC00AE0A3C302E06031D0C2E0630B80089
:100C0000B7019C263508C9003608CA00AE01CB01E1
:100C1000CC01831203134B15831203130430BB0062
:100C200006160000861600002426831603133608D5
:100C3000C6003508C500831203134B14083C031C7F
:100C40004B1000004B130800831203133426630873
:100C500083160313B500831203136208831603136C
:100C6000B6008312031308008515F9260613E20166
:100C7000E30185110000861C3B2E00005526043040
:100C8000A700E30D861C6310861863145526A70B76
:100C9000412E0830A700E20D861C621086186214EF
:100CA0005526A70B4B2E85150800000006170000DF
:100CB0000000061300000800831603130310B50C90
:100CC000B60C831603130310B50CB60C080083167C
:100CD00003133708B5073808B6070318B50A080024
:100CE000831603133708B5023808B602031CB50390
:100CF0000800831603133808B6023708031C370FA1
:100D0000B502080083160313BD01BE011030A10017
:100D1000B50CB60C031C922E3708BD073808BE0769
:100D20000318BD0A0310B80DB70DA10B882E3D089E
:100D3000B5003E08B600080083160313BB01BC01D2
:100D40001030A100B60DB50DBC0DBB0D37083B0230
:100D5000031DAC2E38083C02031CB42E3808BC021C
:100D60003708031CB70FBB02BE0DBD0DA10BA22E91
:100D70003D08B5003E08B60008003508803AB300CB
:100D80003708803A3302C62E37083502031DCA2EB3
:100D90003808360208004330AA00AA0BCD2E0800FE
:100DA0000130AA000130AB002030AC00AC0BD62ED5
:100DB000AB0BD62EAA0BD62E08000130AA000130AC
:100DC000AB000530AC00D62E0130AA000130AB00DC
:100DD0001430AC00D62E0130AA000130AB00283010
:100DE000AC00D62E0130AA000130AB00C830AC00F8
:100DF000D62E0130AA000230AB00F330AC00D62E64
:100E00000130AA000830AB00CD30AC00D62E013046
:100E1000AA004F30AB000130AC00D62E0230AA0041
:100E20008730AB006A30AC00D62E0430AA000E30FA
:100E3000AB003830AC00D62E0830AA00A130AB0091
:100E4000DA30AC00D62E1F30AA008530AB0033302C
:100E5000AC00D62E03102030AE00C001C101C2018B
:100E6000C301C401BF0DBE0DBD0DBC0DC40DC30D2E
:100E7000C20DC10DC00DAE0B3E2F592F4430840062
:100E80004E27433084004E27423084004E274130A5
:100E900084004E27403084004E27322F0330000755
:100EA000C500C519800030300007C500C51B800093
:100EB00008000800A200FE309B3E2202A20D831C07
:100EC000FA3E221CA03EA20C0800A2000130220221
:100ED000A20D831CFA3E221CA03EA20C080035087D
:100EE000603C0319080035085A27B500080035088A
:100EF000031908006527B50008003608243C0319CB
:100F0000080036085A27B6000800360803190800FA
:100F10006527B60008003708283C03190800370881
:100F20005A27B70008003708031908006527B700DB
:100F300008003808123C0319080038085A27B8007E
:100F400008003808031908006527B80008003A08A7
:100F5000993C031908003A085A27BA0008003A08D1
:0A0F6000031908006527BA00080015
:02400E00213F50
:1042000054342E3441346334633420343D34203408
:1042100020342034203420342034203420342034FE
:1042200054342E3441346D34623420343D342034DF
:1042300020342034203420342034203420342034DE
:1042400054342E3445347834743420343D3420349E
:1042500020342034203420342034203420342034BE
:10426000543465347334743420342034203420348E
:10427000203420342034203420342034203420349E
:1042800043346F346E347334543441346D34623497
:10429000203420342034203420342034203420347E
:1042A00043346F346E347334543441346334633480
:1042B000203420342034203420342034203420345E
:1042C000523454344334203441344D344A34483425
:1042D0004D3420342B34393437343534333431349D
:1042E00028344334293450342E34463472346534FF
:0E42F00079346534723420343034363400347E
:00000001FF
